:020000040000FA
:020000000428D2
:08000800FF30A200FF30A3004D
:10001000FF30A4008B01A70106303221FF3076218A
:10002000003074210F30722100306A2100306821C5
:100030000130A8000130A9000130AA00A010201151
:10004000A011051C2628A01C28284F28A01C4F28DA
:10005000A010051C2C28A01405184F28851C40282A
:10006000051E39282908E4202B08A9002908562153
:100070003F28290828212B08A900290856214F28A4
:10008000051E49282908AD202B08A900290856215A
:100090004F2829081B212B08A90029085621051DD6
:1000A0005428201D56287D28201D7D282011051D3F
:1000B0005A28201505197D28851D6E28051E6728DC
:1000C0002808E4202B08A80028085F216D282808AC
:1000D00028212B08A80028085F217D28051E7728E5
:1000E0002808AD202B08A80028085F217D282808B3
:1000F0001B212B08A80028085F21071C8228A01DAF
:100100008428AB28A01DAB28A011071C8828A015A7
:100110000718AB28871C9C28051E95282A08E42070
:100120002B08AA002A084D219B282A0828212B08E1
:10013000AA002A084D21AB28051EA5282A08AD20B3
:100140002B08AA002A084D21AB282A081B212B08BE
:10015000AA002A084D212128AC28AB000F30AB059E
:100160002B08083C031DB7280C30AB00E3282B08F4
:100170000C3C031DBE280430AB00E3282B08043CD4
:10018000031DC5280630AB00E3282B08063C031DE1
:10019000CC280230AB00E3282B08023C031DD328F7
:1001A0000330AB00E3282B08033C031DDA280130A1
:1001B000AB00E3282B08013C031DE1280930AB000C
:1001C000E3280830AB000800AB000F30AB052B086C
:1001D000013C031DEE280330AB001A292B08033C19
:1001E000031DF5280230AB001A292B08023C031D21
:1001F000FC280630AB001A292B08063C031D0329F6
:100200000430AB001A292B08043C031D0A290C30CA
:10021000AB001A292B080C3C031D11290830AB0038
:100220001A292B08083C031D18290930AB001A298C
:100230000130AB000800AB002B1C232903102B0C52
:100240000838AB0025290310AB0C0F30AB050800B4
:10025000AB000310AB0D2B1E2F290130AB040F3068
:10026000AB050800A800A9019F30AA00280838297A
:10027000AB00831F3D29A0143E29A010291C422950
:100280008317432983132A0884002B088000A01CAD
:100290004B2983174C2983130800AB002B0EF03930
:1002A000AC0026080F392C04A6006C29AB002B0EDD
:1002B000F039AC0025080F392C04A5006F29AB00DC
:1002C0002B080F39AC002508F0392C04A5006F2944
:1002D000A6006C29A5006F292608870008002508BC
:1002E00086000800A4007829A3007C29A2008029A8
:1002F00024088421870087292308842186008729F0
:10030000220884218500872983160313080083129D
:0403100003130800CB
:02400E00323F3F
:00000001FF
